:0400000002EF26F0F5
:1000080000C019F001C018F00BC017F00CC016F0B2
:100018000DC015F06F0084FF1AF06F0088FF1BF009
:10002800390193AF15D0A3AF13D03C0EB76EB00E05
:10003800B66E1F4A202A000E006E2050005C02E1B6
:100048001F50090803E2BA7601010A853901A39F06
:10005800A3A78BD093A789D084EC24F000C038F0F4
:100068003D01F9AB0FD0F99B010E01011725006E78
:10007800000E1821016E00C017F101C018F16F00C1
:10008800A0F738F03D01F9A70FD0010E010117259F
:10009800006E000E1821016E00C017F101C018F1A2
:1000A80084EC24F000C038F038500D0A0AE03850CB
:1000B8000A0A07E03750000802E136504F0801E30A
:1000C80035D0010E346E000E356E430E3F24E16EBE
:1000D800000E4020E26E6F0087FFE1FF6F008BFF8C
:1000E800E2FFE66A030E0B6E080E0C6E770E0D6EBD
:1000F8000D2EFED70C2EFCD70B2EFAD73901A3A74D
:1001080003D06F00A0F738F093973FC036F040C097
:1001180037F03F6A406A3750000802E136504F080E
:1001280004E2020E346E000E356E1FD0346A356A52
:10013800430E3F24E16E000E4020E26E6F0087FF01
:10014800E1FF6F008BFFE2FF6000E3F0E6FF3FC0D6
:1001580036F040C037F0010E3F24006E000E4020FC
:10016800016E00C03FF001C040F019C000F018C097
:1001780001F017C00BF016C00CF015C00DF06000B0
:0C0188006BF0E1FF60006FF0E2FF11007F
:0C019400000E3D01F9BF010E006E1200CC
:0C01A000000E3D01E1BF010E006E1200D8
:0401AC00F9DF120065
:0401B000F1DF120069
:1001B4000B820BAEE4EF00F003680268016800688C
:0801C4000A360232FF0E1200A0
:0801CC000AAE029E000E1200B3
:1001D400EBDF005202E10000FBD76000C7F5D2FD5F
:0201E400120007
:0E01E600026A016A006A086A036A000E1200CB
:1001F400DDDF005202E10000FBD76000C7F5EAFD35
:020204001200E6
:100206000B840BAE0EEF01F0010E036E026A016A5B
:0A021600006A0A360232FF0E1200E1
:0E022000550E3A01BF6FAA0EBF6FBF811200CC
:08022E0070C171F1E0DF120064
:0802360070C171F1CCDF120070
:0E023E00550E3A01BF6FAA0EBF6FBF9112009E
:10024C000CB068EF01F00CA20EEF02F00E6A000E7B
:10025C0002647FEF01F0F00E0214D8A44AEF01F013
:10026C00023A01380F0B02260138F00B016E0038F0
:10027C000F0B01260038F00B006E08380F0B002610
:10028C000838F00B086E0E84D89002BE63EF01F0B4
:10029C0008360036013602360E2A02BE63EF01F034
:1002AC0008360036013602360E2A02BE63EF01F024
:1002BC0008360036013602360E2A0E50036404EF5F
:1002CC0002F0035E0BBC08AE09EF02F0D880800E82
:1002DC0008640030000E002201220222D8A009EF8F
:1002EC0002F0023201320032034A0EEF02F009EF43
:1002FC0002F001C002F000C001F008C000F0086A72
:10030C00000E0E860264B6EF01F0F00E0214D8A4B3
:10031C009EEF01F0023A01380F0B02260138F00B68
:10032C00016E00380F0B01260038F00B006E0E84A6
:10033C00D89002BE63EF01F00036013602360E2A69
:10034C0002BE63EF01F00036013602360E2A02BE01
:10035C0063EF01F00036013602360E2A63EF01F02E
:10036C0001C002F000C001F0006A000E0E960E886B
:10037C000264E3EF01F0F00E0214D8A4CEEF01F00A
:10038C00023A01380F0B02260138F00B016E0E8475
:10039C00D89002BE63EF01F0013602360E2A02BE7F
:1003AC0063EF01F0013602360E2A02BE63EF01F054
:1003BC00013602360E2A63EF01F001C002F0016A29
:1003CC00000E0E86026413EF02F0F00E0214D8A495
:1003DC00F2EF01F0023A0E84D89002BE63EF01F006
:1003EC0002360E2A02BE63EF01F002360E2A02BE5E
:1003FC0063EF01F002360E2A63EF01F0010E0C6E72
:10040C00FCDE16EF02F0020E0C6EDADE16EF02F0D6
:10041C00040E0C6EC9DE16EF02F0080E0C6EDDDE5B
:02042C001200BC
:08042E0070C171F1D0DE120073
:0804360070C171F1DCDE12005F
:10043E00086A096A000E07620364A7EF02F0025011
:10044E0006180A6E075003267E0ED8A035EF02F06E
:10045E00035ED8B0ABEF02F039EF02F0035ED8A026
:10046E00AFEF02F0028E068E02C00EF001C00BF04E
:10047E0000C00DF0005004026F00D0FF0CF00150D0
:10048E0005026F00D0FF00F06F00CCFF08F00402F1
:10049E00F3500C26F4500822000E00220D500502D7
:1004AE00F3500C26F4500822000E002202500402D3
:1004BE00F3500826F450002202500502016A000E85
:1004CE000122F3500026F45001220D500602F35083
:1004DE000826F4500022026A000E012202220B505E
:1004EE000602F3500026F4500122000E02220E5096
:1004FE000602F3500126F450022202BE8FEF02F0E4
:10050E0008360036013602360306D8B4AFEF02F0D5
:10051E00A2EF02F0D880800E08640030000E002298
:10052E0001220222D8A0A2EF02F0023201320032E2
:10053E00034AABEF02F00AAE029E000EB1EF02F0DC
:10054E00010E4ADEB1EF02F0020E2DDEB1EF02F027
:06055E00040E52DE120043
:080564000B6A0B86FF0E12006A
:10056C000134083609360450085E0550D8A0053C05
:10057C00095E003601360F0E0C6E01340836093652
:10058C00045000A006D0085E0550D8A0053C095EBA
:10059C0005D008260550D8B0053C09260036013692
:1005AC000C2EEBD700B006D0045008260550D8B05E
:0805BC00053C092600001200B5
:1005C4000D6A086A0050D8B4000C04180A6E0ABEFA
:1005D4000D1E0B6A04AE02D0041E042A00AE02D023
:1005E400001E002A005004100A6E0ABE1FD00450D8
:1005F400085E003600340836045008260036060E1D
:100604000C6E00340836045000B0085E00A00826C2
:1006140000360C2EF6D700A008260BB015D00DAE70
:10062400000C001E002A081E082A000C04AE09D083
:1006340000BE04D00050086E006AF1D7006A002A98
:10064400000C001E0B2AD3D7082A0450085CD8A437
:0E065400E6D7086A002A00AEE2D7FF0C1200BB
:10066200086A080E0C6E003408360450085ED8B0D2
:0E06720002D00826D89000360C2EF5D71200C4
:1006800001016C51170802E2006A0FD36D51000A94
:10069000D8A4B1D06F5301E0D2DD60D06000BBF5CB
:1006A00000FAA5D06000BBF501FAA1D06000BBF54F
:1006B00002FA9DD06000BBF503FA99D06000BBF54B
:1006C00004FA95D06000BBF505FA91D06000BBF547
:1006D00006FA8DD06000BBF507FA89D06000BBF543
:1006E00008FA85D06000BBF509FA81D06000BBF53F
:1006F0000AFA7DD06000BBF50BFA79D06000BBF53B
:100700000CFA75D06000BBF50DFA71D06000BBF536
:100710000EFA6DD06000BBF50FFA69D06000BBF532
:1007200010FA65D06000BBF511FA61D06000BBF52E
:1007300012FA5DD06000BBF513FA59D06000BBF52A
:1007400014FA55D06000BBF515FA51D06000BBF526
:1007500016FA4DD06000BBF517FA49D001016C5173
:10076000000A9CE06C51010A9DE06C51020A9EE077
:100770006C51030A9FE06C51040AA0E06C51050A19
:10078000A1E06C51060AA2E06C51070AA3E06C518B
:10079000080AA4E06C51090AA5E06C510A0AA6E017
:1007A0006C510B0AA7E06C510C0AA8E06C510D0AC1
:1007B000A9E06C510E0AAAE06C510F0AABE06C5133
:1007C000100AACE06C51110AADE06C51120AAEE0B7
:1007D0006C51130AAFE06C51140AB0E06C51150A69
:1007E000B1E06C51160AB2E06C51170AB3E0010196
:1007F0006F5301E015DD01016D51010AD8A452D1FA
:100800006F5301E01CDDA4D06000B3F5C0FA45D100
:100810006000B3F5C1FA41D16000B3F5C2FA3DD131
:100820006000B3F5C3FA39D16000B3F5C4FA35D12D
:100830006000B3F5C5FA31D16000B3F5C6FA2DD129
:100840006000B3F5C7FA29D16000B3F5C8FA25D125
:100850006000B3F5C9FA21D16000B3F5CAFA1DD121
:100860006000B3F5CBFA19D16000B3F5CCFA15D11D
:100870006000B3F5CDFA11D16000B3F5CEFA0DD119
:100880006000B3F5CFFA09D16000B3F5D0FA05D115
:100890006000B3F5D1FA01D16000B3F5D2FAFDD012
:1008A0006000B3F5D3FAF9D06000B3F5D4FAF5D00F
:1008B0006000B3F5D5FAF1D06000B3F5D6FAEDD00B
:1008C0006000B3F5D7FAE9D06000B3F5D8FAE5D007
:1008D0006000B3F5D9FAE1D06000B3F5DAFADDD003
:1008E0006000B3F5DBFAD9D06000B3F5DCFAD5D0FF
:1008F0006000B3F5DDFAD1D06000B3F5DEFACDD0FB
:100900006000B3F5DFFAC9D06000B3F5E0FAC5D0F6
:100910006000B3F5E1FAC1D06000B3F5E2FABDD0F2
:100920006000B3F5E3FAB9D06000B3F5E4FAB5D0EE
:100930006000B3F5E5FAB1D06000B3F5E6FAADD0EA
:100940006000B3F5E8FAA9D06000B3F5E9FAA5D0E4
:1009500001016E51000AD8B457D76E51010AD8B4BC
:1009600057D76E51020AD8B457D76E51030AD8B47C
:1009700057D76E51040AD8B457D76E51050AD8B468
:1009800057D76E51060AD8B457D76E51070AD8B454
:1009900057D76E51080AD8B457D76E51090AD8B440
:1009A00057D76E510A0AD8B457D76E510B0AD8B42C
:1009B00057D76E510C0AD8B457D76E510D0AD8B418
:1009C00057D76E510E0AD8B457D76E510F0AD8B404
:1009D00057D76E51100AD8B457D76E51110AD8B4F0
:1009E00057D76E51120AD8B457D76E51130AD8B4DC
:1009F00057D76E51140AD8B457D76E51150AD8B4C8
:100A000057D76E51160AD8B457D76E51170AD8B4B3
:100A100057D76E51180AD8B457D76E51190AD8B49F
:100A200057D76E511A0AD8B457D76E511B0AD8B48B
:100A300057D76E511C0AD8B457D76E511D0AD8B477
:100A400057D76E511E0AD8B457D76E511F0AD8B463
:100A500057D76E51200AD8B457D76E51210AD8B44F
:100A600057D76E51220AD8B457D76E51230AD8B43B
:100A700057D76E51240AD8B457D76E51250AD8B427
:100A800057D76E51260AD8B457D76E51270AD8B413
:100A900057D76E51280AD8B457D701016F5302E0D7
:100AA00010EC01F0A8D001016DB102D0C29001D0CC
:100AB000C280F9D001016DB102D0C29201D0C282D0
:100AC000F2D001016DB102D0C29401D0C284EBD04A
:100AD00001016DB102D0C29601D0C286E4D00101FD
:100AE0006DB102D0C29801D0C288DDD001016DB1D4
:100AF00002D0C29A01D0C28AD6D001016DB102D013
:100B0000C29C01D0C28CCFD001016DB102D0C29E77
:100B100001D0C28EC8D001016DB102D0C39001D006
:100B2000C380C1D001016DB102D0C39201D0C38294
:100B3000BAD001016DB102D0C39401D0C384B3D047
:100B400001016DB102D0C39601D0C386ACD00101C2
:100B50006DB102D0C39801D0C388A5D001016DB199
:100B600002D0C39A01D0C38A9ED001016DB102D0D8
:100B7000C39C01D0C38C97D001016DB102D0C39E3C
:100B800001D0C38E90D001016DB102D0C49001D0CC
:100B9000C48089D001016DB102D0C49201D0C48259
:100BA00082D001016DB102D0C49401D0C4847BD045
:100BB00001016DB102D0C49601D0C48674D0010188
:100BC0006DB102D0C49801D0C4886DD001016DB15F
:100BD00002D0C49A01D0C48A66D001016DB102D09E
:100BE000C49C01D0C48C5FD001016DB102D0C49E01
:100BF00001D0C48E58D001016C51000AD8B453D72B
:100C00006C51010AD8B456D76C51020AD8B459D7DE
:100C10006C51030AD8B45CD76C51040AD8B45FD7BE
:100C20006C51050AD8B462D76C51060AD8B465D79E
:100C30006C51070AD8B468D76C51080AD8B46BD77E
:100C40006C51090AD8B46ED76C510A0AD8B471D75E
:100C50006C510B0AD8B474D76C510C0AD8B477D73E
:100C60006C510D0AD8B47AD76C510E0AD8B47DD71E
:100C70006C510F0A81E06C51100A85E06C51110A29
:100C800089E06C51120A8DE06C51130A91E06C51AD
:100C9000140A95E06C51150A99E06C51160A9DE012
:0C0CA0006C51170AA1E0FF0E006E12005C
:100CAC000B800BAE62EF06F0026A0AAEFF0E026E0C
:0C0CBC00016E006E0A360232FF0E1200BC
:100CC800025006180E6E086A096A0B6A0350076418
:100CD80057EF07F006500A6E068E028E03500B6E11
:100CE8000750036E000E0B64A7EF06F00B50075E6B
:100CF800D8B448EF07F0070E076416EF07F0075E51
:100D080000C008F001C000F002C001F0026A074EFE
:100D180048EF07F00764EBEF06F0075E00C008F045
:100D280001C000F0016A074E48EF07F00764C9EFF9
:100D380006F0075E00C008F0006A074E48EF07F0AB
:100D48000764B0EF06F00AC002F005C001F004C065
:100D580000F0086A74EF08F0030E0764BBEF06F0B2
:100D6800075E08380F0B086E074E48EF07F0D8905B
:100D78000832074E48EF07F0D8900832074E48EF80
:100D880007F0D890083248EF07F0030E0764DAEF4F
:100D980006F0075E08380F0B086E0038F00B0826BF
:100DA80000380F0B006E074E48EF07F0D89000325E
:100DB8000832074E48EF07F0D89000320832074E45
:100DC80048EF07F0D8900032083248EF07F0030EDA
:100DD800076402EF07F0075E08380F0B086E00384B
:100DE800F00B082600380F0B006E0138F00B0026B8
:100DF80001380F0B016E074E48EF07F0D89001320B
:100E080000320832074E48EF07F0D890013200321E
:100E18000832074E48EF07F0D89001320032083206
:100E280048EF07F0030E076433EF07F0075E083852
:100E38000F0B086E0038F00B082600380F0B006EF9
:100E48000138F00B002601380F0B016E0238F00B49
:100E5800012602380F0B026E074E48EF07F0D890B4
:100E68000232013200320832074E48EF07F0D890BC
:100E78000232013200320832074E48EF07F0D890AC
:100E88000232013200320832096A000E0EAE3CEF1F
:100E980008F0081E001E011E021E082A0022012258
:100EA80002223CEF08F00750D8A45DEF07F074EF7A
:100EB80008F0096A02C00AF0028E068E0750035C29
:100EC800076ED8B42FEF08F0070E0764FDEF07F0A0
:100ED800075E0450096E0550046E0650056E066ADA
:100EE800074E2FEF08F0070E0764D2EF07F0075EF2
:100EF8000450096E0550046E056A074E2FEF08F07E
:100F0800070E0764B0EF07F0075E0450096E046A25
:100F1800074E2FEF08F0070E076497EF07F00AC097
:100F280002F074EF08F0030E0764A2EF07F0075E03
:100F380009380F0B096E074E2FEF08F0D8900932C9
:100F4800074E2FEF08F0D8900932074E2FEF08F020
:100F5800D89009322FEF08F0030E0764C1EF07F0AD
:100F6800075E09380F0B096E0438F00B09260438A0
:100F78000F0B046E074E2FEF08F0D8900432093299
:100F8800074E2FEF08F0D89004320932074E2FEFA2
:100F980008F0D890043209322FEF08F0030E0764E6
:100FA800E9EF07F0075E09380F0B096E0438F00BFC
:100FB800092604380F0B046E0538F00B0426053893
:100FC8000F0B056E074E2FEF08F0D890053204324C
:100FD8000932074E2FEF08F0D89005320432093253
:100FE800074E2FEF08F0D8900532043209322FEF60
:100FF80008F0030E07641AEF08F0075E09380F0BB4
:10100800096E0438F00B092604380F0B046E0538F6
:10101800F00B042605380F0B056E0638F00B052675
:1010280006380F0B066E074E2FEF08F0D8900632E1
:10103800053204320932074E2FEF08F0D8900632F5
:10104800053204320932074E2FEF08F0D8900632E5
:10105800053204320932086A000E0EAE3CEF08F081
:10106800091E041E051E061E092A04220522062240
:101078000950082604500022055001220650022279
:101088000EBE53EF08F0D8A062EF08F0023201322A
:1010980000320832033E62EF08F06EEF08F0D8B075
:1010A80068EF08F0000E081E001E011E021E082A26
:1010B8000022012202220A7E68EF08F0010E0C6E5F
:1010C80026EC01F076EF08F0020E0C6E26EC01F02B
:1010D80076EF08F0040E0C6EDAEC00F076EF08F00C
:0610E800000E0C6E120068
:1010EE00D250026ED29E0500FF6A0150FE6E005075
:0810FE00FD6E02BED28E12004D
:1011060003500718D8A497EF08F002500618D8A481
:1011160097EF08F001500518D8A497EF08F0005093
:0E1126000418D8B4D8841200D8941200120015
:101134000450000A08E10550000A05E1FF0E006EA4
:101144007F0E016E58D00D6A096A086A01500010BA
:10115400D8B4000C015005180A6E0ABE0D1E0B6AA5
:1011640005AE05D0041E051E042AD8B4052A01AE16
:1011740005D0001E011E002AD8B4012A0150051012
:101184000A6E0ABE10D0B6EC02F00BB020D00DAE41
:10119400000C001E011E002AD8B4012A081E091ED4
:1011A400082AD8B4092A000C05AE0DD001BE07D018
:1011B4000150096E0050086E016A006AE8D7016A9E
:1011C400006A002A000C011E001E0B2ADDD7082A23
:1011D400D8B4092A0450085CD8A4D9D70550095CAE
:1011E400D8A4D5D7096A086A002AD8B4012A01AE5E
:0811F400CED70000FF0C120031
:1011FC00800E01016719006E800E000A005CD8B0E9
:10120C0085D167510008016E01C067F1800E01188D
:10121C00006E800E6E0A005CD8A0CCD0640E046EFA
:10122C0067C100F0E2EC02F0120E0024056E000E15
:10123C0000BEFF0E066E000E062205C000F006C0B2
:10124C0001F0000E06BEFF0E026E036E003600901B
:10125C00013602360336003600900136023603366C
:10126C00B10E0024F66E570E0120F76E000E022010
:10127C00F86E09006F00D4FF68F109006F00D4FF0D
:10128C0069F109006F00D4FF6AF109006F00D4FF07
:10129C006BF1640E046E67C100F0E2EC02F008C062
:1012AC0000F00A0E046EE2EC02F0090E0024056E4A
:1012BC00000E00BEFF0E066E000E062205C000F0EA
:1012CC0006C001F0000E06BEFF0E026E036E003665
:1012DC000090013602360336003600900136023695
:1012EC000336B10E0024F66E570E0120F76E000E79
:1012FC000220F86E09006F00D4FF00F009006F00A7
:10130C00D4FF01F009006F00D4FF02F009006F0058
:10131C00D4FF03F068C104F069C105F06AC106F09E
:10132C006BC107F01FEC02F000C068F101C069F15D
:10133C0002C06AF103C06BF10A0E046E67C100F0C3
:10134C00E2EC02F008C000F000C001F0000E00BE9C
:10135C00FF0E026E036E046E0136019002360336E8
:10136C00043601360190023603360436B10E0124E0
:10137C00F66E570E0220F76E000E0320F86E090071
:10138C006F00D4FF00F009006F00D4FF01F00900DA
:10139C006F00D4FF02F009006F00D4FF03F068C1A6
:1013AC0004F069C105F06AC106F06BC107F01FECCF
:1013BC0002F02BD2800E0A0A006E800E6719005CB8
:1013CC0079E20A0E046E67C100F0E2EC02F0090E3D
:1013DC000024056E000E00BEFF0E066E000E0622E7
:1013EC0005C000F006C001F0000E06BEFF0E026E36
:1013FC00036E00360090013602360336003600903C
:10140C00013602360336B10E0024F66E570E01205B
:10141C00F76E000E0220F86E09006F00D4FF68F121
:10142C0009006F00D4FF69F109006F00D4FF6AF165
:10143C0009006F00D4FF6BF10A0E046E67C100F057
:10144C00E2EC02F008C000F000C001F0000E00BE9B
:10145C00FF0E026E036E046E0136019002360336E7
:10146C00043601360190023603360436B10E0124DF
:10147C00F66E570E0220F76E000E0320F86E090070
:10148C006F00D4FF00F009006F00D4FF01F00900D9
:10149C006F00D4FF02F009006F00D4FF03F068C1A5
:1014AC0004F069C105F06AC106F06BC107F01FECCE
:1014BC0002F0ABD167C100F0000E67BFFF0E016EEA
:1014CC00026E036E0036009001360236033600368B
:1014DC000090013602360336B10E0024F66E570E1C
:1014EC000120F76E000E0220F86E09006F00D4FF89
:1014FC0000F009006F00D4FF01F009006F00D4FF69
:10150C0002F009006F00D4FF03F07FD1800E671941
:10151C00006E800E6E0A005CD8A0CCD0640E046EF7
:10152C0067C100F0E2EC02F0120E0024056E000E12
:10153C0000BEFF0E066E000E062205C000F006C0AF
:10154C0001F0000E06BEFF0E026E036E0036009018
:10155C000136023603360036009001360236033669
:10156C00E50E0024F66E570E0120F76E000E0220D9
:10157C00F86E09006F00D4FF68F109006F00D4FF0A
:10158C0069F109006F00D4FF6AF109006F00D4FF04
:10159C006BF1640E046E67C100F0E2EC02F008C05F
:1015AC0000F00A0E046EE2EC02F0090E0024056E47
:1015BC00000E00BEFF0E066E000E062205C000F0E7
:1015CC0006C001F0000E06BEFF0E026E036E003662
:1015DC000090013602360336003600900136023692
:1015EC000336E50E0024F66E570E0120F76E000E42
:1015FC000220F86E09006F00D4FF00F009006F00A4
:10160C00D4FF01F009006F00D4FF02F009006F0055
:10161C00D4FF03F068C104F069C105F06AC106F09B
:10162C006BC107F01FEC02F000C068F101C069F15A
:10163C0002C06AF103C06BF10A0E046E67C100F0C0
:10164C00E2EC02F008C000F000C001F0000E00BE99
:10165C00FF0E026E036E046E0136019002360336E5
:10166C00043601360190023603360436E50E0124A9
:10167C00F66E570E0220F76E000E0320F86E09006E
:10168C006F00D4FF00F009006F00D4FF01F00900D7
:10169C006F00D4FF02F009006F00D4FF03F068C1A3
:1016AC0004F069C105F06AC106F06BC107F01FECCC
:1016BC0002F0ABD0800E0A0A006E800E6719005C37
:1016CC0079E20A0E046E67C100F0E2EC02F0090E3A
:1016DC000024056E000E00BEFF0E066E000E0622E4
:1016EC0005C000F006C001F0000E06BEFF0E026E33
:1016FC00036E003600900136023603360036009039
:10170C00013602360336E50E0024F66E570E012024
:10171C00F76E000E0220F86E09006F00D4FF68F11E
:10172C0009006F00D4FF69F109006F00D4FF6AF162
:10173C0009006F00D4FF6BF10A0E046E67C100F054
:10174C00E2EC02F008C000F000C001F0000E00BE98
:10175C00FF0E026E036E046E0136019002360336E4
:10176C00043601360190023603360436E50E0124A8
:10177C00F66E570E0220F76E000E0320F86E09006D
:10178C006F00D4FF00F009006F00D4FF01F00900D6
:10179C006F00D4FF02F009006F00D4FF03F068C1A2
:1017AC0004F069C105F06AC106F06BC107F01FECCB
:1017BC0002F02BD067C100F0000E67BFFF0E016E68
:1017CC00026E036E00360090013602360336003688
:1017DC000090013602360336E50E0024F66E570EE5
:1017EC000120F76E000E0220F86E09006F00D4FF86
:1017FC0000F009006F00D4FF01F009006F00D4FF66
:0C180C0002F009006F00D4FF03F012008E
:101818000A6A0350D8A40A800750D8A40A820A503A
:10182800D8B46FEF0CF0030AD8B428EF0CF00AB064
:1018380023EF0CF006AE6DEF0CF06BEF0CF002AE80
:101848006BEF0CF06DEF0CF00250800B0A6E029EED
:101858000650800B069E0A18D8B439EF0CF00A50CF
:10186800D8B46BEF0CF06DEF0CF00750035CD8B4F4
:1018780043EF0CF0D8A05FEF0CF065EF0CF00650CA
:10188800025CD8B44DEF0CF0D8A05FEF0CF065EF18
:101898000CF00550015CD8B457EF0CF0D8A05FEFFE
:1018A8000CF065EF0CF00450005CD8B46FEF0CF04E
:1018B800D8B065EF0CF00A52D8B46DEF0CF06BEFAE
:1018C8000CF00A52D8B46BEF0CF06DEF0CF0D88026
:0E18D8001200D8901200D880D884120012009E
:1018E60001016751390806E3300E675D03E3010E17
:0818F600006E01D0006A12002F
:1018FE000B6A0A6A096A005004026F00D0FF09F0F1
:10190E006F00CCFF08F0015005026F00D0FF0BF006
:10191E006F00CCFF0AF000500502F3500926F45078
:10192E000A22E86A0B2201500402F3500926F450F1
:10193E000A22E86A0B2208C000F009C001F00AC0B2
:08194E0002F00BC003F01200CF
:1019560060007FF4E1FF600083F4E2FF60009FF522
:10196600E6FF1DC100F01EC101F077EC08F0120081
:101976000450000A12E10550000A0FE10650000A61
:101986000CE10750000A09E1FF0E006EFF0E016E22
:101996007F0E026EFF0E036EA8D0086A096A075012
:1019A600D8B466EF0DF00350D8B46BEF0DF00250CB
:1019B60006180A6E028E068E0E6A02C008F001C074
:1019C6000CF000C00DF004500D5E0550D8A0053C8B
:1019D6000C5E0650D8A0063C085E086A0C6A0D6AC2
:1019E600D8A0FDEF0CF0D890023201320032083256
:1019F600010E0E6E0750035ED8A00AEF0DF07E0EA4
:101A06000E240326D8B070EF0DF010EF0DF07E0E09
:101A16000E240326D8A075EF0DF0180E0B6E0D36AA
:101A26000C3608360036013602360E360450005E95
:101A36000550D8A0053C015E0650D8A0063C025EC3
:101A460006340E120EA02BEF0DF00D8036EF0DF0C2
:101A5600045000260550D8B0053C01260650D8B0E3
:101A6600062802260D900B2E12EF0DF05CEF0DF0FE
:101A7600D8900036013602360E360450005E055008
:101A8600D8A0053C015E0650D8A0063C025E06348E
:101A96000E10010B0D26D8B00C2AD8B4082AD8A4EB
:101AA6005CEF0DF008320C320D32032AD8B470EF19
:101AB6000DF00AAE089E0850026E0C50016E0D50D5
:101AC600006E78EF0DF0010EB2EC02F078EF0DF03B
:101AD600020EF3EC00F078EF0DF0040EDAEC00F0F5
:0C1AE60078EF0DF0080E03EC01F0120088
:0C1AF2003A0E0D6E0D2EFED70000120003
:101AFE000B6A0C6A086A0350D8B403EF0EF002C0EA
:101B0E000AF0028E9E0E035E03AEF3EF0DF0036C31
:101B1E00080E035CD8A0C0EF0DF0036E083600C0AF
:101B2E0008F001C000F002C001F0026A080E035C6A
:101B3E00D8A0C0EF0DF0036E083600C008F001C04B
:101B4E0000F0016A080E035CD8A0C0EF0DF0036E22
:101B5E00083600C008F0006A080E035CD8A0C0EF7B
:101B6E000DF0036E0836086A0350D8A4D890CCEF57
:101B7E000DF00350D8B4CCEF0DF0D89002320132F4
:101B8E0000320832032EC4EF0DF00BBC08A0DDEFBF
:101B9E000DF0D8A0DDEF0DF0082AD8B4002AD8B485
:101BAE00012AD8B4022A02BE07EF0EF00AAE03EFE6
:101BBE000EF0021E011E001E081E082AD8B4002AAE
:101BCE00D8B4012AD8B4022A03EF0EF0026A016AD1
:101BDE00006A086A03EF0EF00B800BAE0EEF0EF0EC
:101BEE00026A0AAE0EEF0EF0026E016E006E086E05
:101BFE000A3602320EEF0EF00C6A000E0FEF0EF0E8
:101C0E00010E0C6E000E56EC06F00FEF0EF0FF0EEE
:101C1E000250036E0150026E0050016E0850006EAD
:021C2E001200A2
:101C30000B6A0A6A096A086A0E6A03340836045095
:101C4000085E0550D8A0053C095E0650D8A0063CA9
:101C50000A5E0750D8A0073C0B5EE86AD8A0010EC8
:101C60000E5E0336070E0C6E0334083609360A364C
:101C70000B360E36045003A012D0085E0550D8A0D3
:101C8000053C095E0650D8A0063C0A5E0750D8A065
:101C9000073C0B5EE86AD8A0010E0E5E11D0082644
:101CA0000550D8B0053C09260650D8B0063C0A2697
:101CB0000750D8B0073C0B26E86AD8B0010E0E26B4
:101CC00003360C2ED1D70234083609360A360B36C5
:101CD0000E36045003A012D0085E0550D8A0053C73
:101CE000095E0650D8A0063C0A5E0750D8A0073C03
:101CF0000B5EE86AD8A0010E0E5E11D008260550D2
:101D0000D8B0053C09260650D8B0063C0A26075034
:101D1000D8B0073C0B26E86AD8B0010E0E26023672
:101D2000070E0C6E0234083609360A360B360E36AC
:101D3000045002A012D0085E0550D8A0053C095EF0
:101D40000650D8A0063C0A5E0750D8A0073C0B5EA0
:101D5000E86AD8A0010E0E5E11D008260550D8B052
:101D6000053C09260650D8B0063C0A260750D8B0D4
:101D7000073C0B26E86AD8B0010E0E2602360C2E60
:101D8000D1D70134083609360A360B360E360450E0
:101D900002A012D0085E0550D8A0053C095E06508E
:101DA000D8A0063C0A5E0750D8A0073C0B5EE86A44
:101DB000D8A0010E0E5E11D008260550D8B0053C03
:101DC00009260650D8B0063C0A260750D8B0073C72
:101DD0000B26E86AD8B0010E0E260136070E0C6EEF
:101DE0000134083609360A360B360E36045001A087
:101DF00012D0085E0550D8A0053C095E0650D8A058
:101E0000063C0A5E0750D8A0073C0B5EE86AD8A0E3
:101E1000010E0E5E11D008260550D8B0053C0926EB
:101E20000650D8B0063C0A260750D8B0073C0B260F
:101E3000E86AD8B0010E0E2601360C2ED1D7003438
:101E4000083609360A360B360E36045001A012D079
:101E5000085E0550D8A0053C095E0650D8A0063C97
:101E60000A5E0750D8A0073C0B5EE86AD8A0010EB6
:101E70000E5E11D008260550D8B0053C0926065044
:101E8000D8B0063C0A260750D8B0073C0B26E86AB3
:101E9000D8B0010E0E260036070E0C6E0034083640
:101EA00009360A360B360E36045000A012D0085EF2
:101EB0000550D8A0053C095E0650D8A0063C0A5E35
:101EC0000750D8A0073C0B5EE86AD8A0010E0E5E52
:101ED00011D008260550D8B0053C09260650D8B0C8
:101EE000063C0A260750D8B0073C0B26E86AD8B053
:101EF000010E0E2600360C2ED1D700B00ED00450A5
:101F000008260550D8B0053C09260650D8B0063C36
:0C1F10000A260750D8B0073C0B26120030
:101F1C006E0E0101675DD8A0D6D0640E046E67C149
:101F2C0000F031EC03F0120E0024056E066A000E70
:101F3C00062205C000F006C001F0000E06BEFF0E22
:101F4C00026E036E00360090013602360336003600
:101F5C000090013602360336B10E0024F66E570E91
:101F6C000120F76E000E0220F86E09006F00D4FFFE
:101F7C0000F009006F00D4FF01F009006F00D4FFDE
:101F8C0002F009006F00D4FF03F0000E046E000E87
:101F9C00056E000E066E7E0E076E1FEC02F000C082
:101FAC0068F101C069F102C06AF103C06BF1640E03
:101FBC00046E67C100F031EC03F008C000F00A0EAB
:101FCC00046E31EC03F0090E0024056E066A000E57
:101FDC00062205C000F006C001F0000E06BEFF0E82
:101FEC00026E036E00360090013602360336003660
:101FFC000090013602360336B10E0024F66E570EF1
:10200C000120F76E000E0220F86E09006F00D4FF5D
:10201C0000F009006F00D4FF01F009006F00D4FF3D
:10202C0002F009006F00D4FF03F068C104F069C12D
:10203C0005F06AC106F06BC107F01FEC02F000C09E
:10204C0068F101C069F102C06AF103C06BF10A0EBC
:10205C00046E67C100F031EC03F008C000F000C062
:10206C0001F0000E026E036E046E01360190023612
:10207C000336043601360190023603360436B10EAF
:10208C000124F66E570E0220F76E000E0320F86E38
:10209C0009006F00D4FF00F009006F00D4FF01F0BD
:1020AC0009006F00D4FF02F009006F00D4FF03F0A9
:1020BC0068C104F069C105F06AC106F06BC107F094
:1020CC001FEC02F0BDD067510A08D8B086D00A0EBA
:1020DC00046E67C100F031EC03F0090E0024056EAC
:1020EC00066A000E062205C000F006C001F0000EC4
:1020FC0006BEFF0E026E036E0036009001360236ED
:10210C00033600360090013602360336B10E002439
:10211C00F66E570E0120F76E000E0220F86E0900C5
:10212C006F00D4FF00F009006F00D4FF01F009002C
:10213C006F00D4FF02F009006F00D4FF03F0000E13
:10214C00046E000E056E000E066E7E0E076E1FEC02
:10215C0002F000C068F101C069F102C06AF103C06D
:10216C006BF10A0E046E67C100F031EC03F008C08D
:10217C0000F000C001F0000E026E036E046E01361A
:10218C0001900236033604360136019002360336CE
:10219C000436B10E0124F66E570E0220F76E000EB7
:1021AC000320F86E09006F00D4FF00F009006F00E7
:1021BC00D4FF01F009006F00D4FF02F009006F009A
:1021CC00D4FF03F068C104F069C105F06AC106F0E0
:1021DC006BC107F01FEC02F033D067C100F0000EAA
:1021EC00016E026E036E0036009001360236033625
:1021FC0000360090013602360336B10E0024F66E1E
:10220C00570E0120F76E000E0220F86E09006F00C9
:10221C00D4FF00F009006F00D4FF01F009006F003B
:10222C00D4FF02F009006F00D4FF03F0000E046E1F
:10223C00000E056E000E066E7E0E076E1FEC02F091
:02224C0012007E
:08224E00067E64EC06F01200AC
:1022560067C16CF168C16DF169C16EF1010E0101D2
:082266006F6F40EC03F0120061
:10226E000B6A0C6A0A6A086A0350D8B4BFEF11F001
:10227E00028E9E0E035E03BE4AEF11F0D8B44AEFF3
:10228E0011F0AFEF11F0036C080E035CD8A07CEFD9
:10229E0011F0036E083600C008F001C000F002C055
:1022AE0001F0026A080E035CD8A07CEF11F0036EF9
:1022BE00083600C008F001C000F0016A080E035C89
:1022CE00D8A07CEF11F0036E083600C008F0006A4B
:1022DE00080E035CD8A07CEF11F0036E0836086A76
:1022EE000350D8A4D89088EF11F00350D8B488EFDB
:1022FE0011F0D8900232013200320832032E80EFF4
:10230E0011F00BBC08A099EF11F0D8A099EF11F0C5
:10231E00082AD8B4002AD8B4012AD8B4022A02BE98
:10232E00C3EF11F00AAEBFEF11F0021E011E001E28
:10233E00081E082AD8B4002AD8B4012AD8B4022A12
:10234E00BFEF11F0026A016A006A086ABFEF11F06E
:10235E000B800BAEC9EF11F0026A0AAEC9EF11F095
:10236E00026E016E006E086E0A360232C9EF11F06F
:10237E00000E0C6ACAEF11F0010E0C6E56EC06F050
:10238E00CAEF11F0FF0E0250036E0150026E0050A4
:08239E00016E0850006E1200F0
:1023A6000050086E0150006E0250016E0350026E1E
:1023B600036A0B6A0C6A9E0E036E0A6A020E0C6EA4
:0623C60026EC01F01200FC
:1023CC0001013F510308D8A03F6B40510308D8A02E
:1023DC00406BF00E3D01F21701013F513D01F2132C
:1023EC00300EF21340C100F0003600900036009021
:1023FC0000360090003600900050F413F38F12005A
:10240C0001015F6B606B536B546B41C100F042C1B7
:10241C0001F043C102F0010E4127000E4223432379
:10242C00600003F0F6FF600007F0F7FF60000BF0B0
:10243C00F8FF09006F00D4FF00F000C050F100520B
:10244C00D8B485EF23F05051250A0EE06000FFF45C
:10245C00E1FF600003F5E2FF600043F5E6FF3F4B50
:10246C00402B5F4B602BD1D7516B526B536B546B22
:10247C0023D05387010E4127000E422343236DD0F6
:10248C005381010E4127000E4223432366D0538310
:10249C00010E4127000E422343235FD05487010EC7
:1024AC004127000E4223432358D05385010E412768
:1024BC00000E4223432351D0600007F5F6FF600065
:1024CC000BF5F7FF60000FF5F8FF09006F00D4FF64
:1024DC0001F001502D0ACDE0600007F5F6FF600019
:1024EC000BF5F7FF60000FF5F8FF09006F00D4FF44
:1024FC0001F00150200AC4E0600007F5F6FF60000F
:10250C000BF5F7FF60000FF5F8FF09006F00D4FF23
:10251C0001F001502B0ABBE0600007F5F6FF6000EC
:10252C000BF5F7FF60000FF5F8FF09006F00D4FF03
:10253C0001F00150230AB2E0600007F5F6FF6000DD
:10254C000BF5F7FF60000FF5F8FF09006F00D4FFE3
:10255C0001F00150300AA9E001D08AD753A301D071
:10256C00539153A701D05395600007F5F6FF600017
:10257C000BF5F7FF60000FF5F8FF09006F00D4FFB3
:10258C0000F0000E016E00C067F173EC0CF000520D
:10259C003EE0516B526B51C100F052C101F00A0E7A
:1025AC00046E000E056E7FEC0CF0600007F5F6FF74
:1025BC0060000BF5F7FF60000FF5F8FF09006F00E6
:1025CC00D4FF02F002500024516F000E0120526F14
:1025DC00300E515F000E525B010E4127000E42235C
:1025EC004323600007F5F6FF60000BF5F7FF600072
:1025FC000FF5F8FF09006F00D4FF00F0000E016E1C
:10260C0000C067F173EC0CF00052C5E145D06000DE
:10261C0007F5F6FF60000BF5F7FF60000FF5F8FF0C
:10262C0009006F00D4FF01F001502A0A35E1600067
:10263C0013F5E9FF600017F5EAFF6F00B8FF00F033
:10264C006F00B8FF01F0600003F0E9FF600007F0D5
:10265C00EAFF6F00B8FF51F16F00B8FF52F1600054
:10266C0013F5E9FF600017F5EAFF020EEE24006E89
:10267C00000EEE20016E600013F5E1FF600017F50F
:10268C00E2FF600003F0E6FF600007F0E6FF010EDA
:10269C004127000E42234323600007F5F6FF60003C
:1026AC000BF5F7FF60000FF5F8FF09006F00D4FF82
:1026BC0001F001502E0AD8A48AD0010E4127000E39
:1026CC0042234323600007F5F6FF60000BF5F7FF8C
:1026DC0060000FF5F8FF09006F00D4FF01F0015006
:1026EC002A0A36E1600013F5E9FF600017F5EAFFEE
:1026FC006F00B8FF00F06F00B8FF01F0600003F04E
:10270C00E9FF600007F0EAFF6F00B8FF4EF16F00C1
:10271C00B8FF4FF1600013F5E9FF600017F5EAFF11
:10272C00020EEE24006E000EEE20016E600013F51A
:10273C00E1FF600017F5E2FF600003F0E6FF6000C8
:10274C0007F0E6FF010E4127000E422343233ED043
:10275C004E6B4F6B600007F5F6FF60000BF5F7FF53
:10276C0060000FF5F8FF09006F00D4FF00F0000EB9
:10277C00016E00C067F173EC0CF0005227E04EC103
:10278C0000F04FC101F00A0E046E000E056E7FECD6
:10279C000CF0600007F5F6FF60000BF5F7FF60002A
:1027AC000FF5F8FF09006F00D4FF02F0025000246F
:1027BC004E6F000E01204F6F300E4E5F000E4F5BC0
:1027CC00010E4127000E42234323C4D703D04E6B86
:1027DC004F6B548941C100F042C101F043C102F07A
:1027EC00010E4127000E42234323600003F0F6FF45
:1027FC00600007F0F7FF60000BF0F8FF09006F00B6
:10280C00D4FF50F11DD15FC100F060C101F089EF20
:10281C0023F05389DFD7548552D1538B54814FD138
:10282C0054834DD1538D4BD14AD1538B538F47D1B8
:10283C00600013F5E9FF600017F5EAFF6F00B8FFC1
:10284C0000F06F00B8FF01F0600003F0E9FF6000DA
:10285C0007F0EAFF6F00B8FF5BF16F00B8FF5CF1A7
:10286C00600013F5E9FF600017F5EAFF020EEE2495
:10287C00006E000EEE20016E600013F5E1FF6000AB
:10288C0017F5E2FF600003F0E6FF600007F0E6FFDB
:10289C00000E5C1902E1000E5B1904E1210E5B6F66
:1028AC00000E5C6F5D6B5E6B5D515B25E96E5E517E
:1028BC005C21EA6EEE520BE0010E5D25006E000EFF
:1028CC005E21016E00C05DF101C05EF1EDD74E518D
:1028DC004F110AE05E514F5D02E15D514E5D04E225
:1028EC004EC15DF14FC15EF152515E5D02E151513D
:1028FC005D5D05E25D51515F5E51525B02D0516BE3
:10290C00526B53B718D051C100F052C101F0010EF7
:10291C00515F000E525B005001100DE06000FFF49F
:10292C00E1FF600003F5E2FF200EE66E3F4B402B0B
:10293C005F4B602BE8D75DC102F05EC103F0010E66
:10294C005D5D006E000E5E59016E00C05DF101C050
:10295C005EF1025003101EE060006FF5E9FF6000AD
:10296C0073F5EAFF6000FFF4E1FF600003F5E2FF9E
:10297C006F00BBFFE6FF3F4B402B010E5B25006E4B
:10298C00000E5C21016E00C05BF101C05CF15F4B7D
:10299C00602BD1D753A718D051C100F052C101F010
:1029AC00010E515F000E525B005001100DE06000F3
:1029BC00FFF4E1FF600003F5E2FF200EE66E3F4BF3
:1029CC00402B5F4B602BE8D720D5600013F5E9FF57
:1029DC00600017F5EAFF6F00B8FF00F06F00B8FF5A
:1029EC0001F0600003F0E9FF600007F0EAFF6F0000
:1029FC00B8FF50F1600013F5E9FF600017F5EAFF2E
:102A0C00020EEE24006E000EEE20016E600013F537
:102A1C00E1FF600017F5E2FF600003F0E6FF6000E5
:102A2C0007F0E6FF500E5B6F010E5C6F010E5D6FE1
:102A3C00000E5E6F4CD7C00E5313000E54133FD0D4
:102A4C005051000AD8B4DFD650516C0AD8B4E1D634
:102A5C0050514C0AD8B4DDD65051660AD8B4DBD6E6
:102A6C005051450AD8B4D9D65051650AD8B4D6D6E7
:102A7C005051670AD8B4D4D650516F0AD8B4D2D6B4
:102A8C005051640AD8B4D0D65051690AD8B4CCD6B7
:102A9C005051700AD8B4C9D65051580AD8B4C5D6BA
:102AAC005051780AD8B4C2D65051730AD8B4C0D693
:102ABC005051630A8AE05051750ABDE0B3D7000E3D
:102ACC005315006E5451070B016E00500110D8B411
:102ADC00B0EF1EF054A904D0060E4E6F000E4F6FCF
:102AEC00600013F5E9FF600017F5EAFF6F00B8FF0F
:102AFC0000F06F00B8FF01F0600003F0E9FF600028
:102B0C0007F0EAFF6F00B8FF55F16F00B8FF56F100
:102B1C006F00B8FF57F16F00B8FF58F1600013F564
:102B2C00E9FF600017F5EAFF040EEE24006E000EBC
:102B3C00EE20016E600013F5E1FF600017F5E2FF77
:102B4C00600003F0E6FF600007F0E6FF046A056A28
:102B5C00066A076A55C100F056C101F057C102F070
:102B6C0058C103F00CEC0CF0010ED8B0000E006E46
:102B7C00005205E0577F030E5313000E5413596B8C
:102B8C005A6B55C100F056C101F057C102F058C143
:102B9C0003F0046A056A066A076A83EC08F0000E03
:102BAC00D8A4010E006E0052D8B48AD058C100F0DF
:102BBC00016A026A036AFF0E0016000E01167E0EF1
:102BCC00005E000E015A00C059F101C05AF1010E0D
:102BDC00005E000E015A00C059F101C05AF1030EFB
:102BEC00046E000E056E7FEC0CF000C059F101C0B4
:102BFC005AF10A0E046E000E056E9AEC08F000C035
:102C0C0059F101C05AF1800E0118026E800E025C5F
:102C1C0002E1000E005C05E2010E0101595F000E9D
:102C2C005A5B010159510008676FFEEC08F055C161
:102C3C0004F056C105F057C106F058C107F01FEC5F
:102C4C0002F000C05BF101C05CF102C05DF103C099
:102C5C005EF1000E046E000E056E000E066E7F0E09
:102C6C00076E5BC100F05CC101F05DC102F05EC19A
:102C7C0003F00CEC0CF0010ED8B0000E006E0052FC
:102C8C0005E0010E595F000E5A5B1AD0000E046E5F
:102C9C00000E056E200E066E820E076E5BC100F0F4
:102CAC005CC101F05DC102F05EC103F00CEC0CF0F4
:102CBC00000ED8B0010E006E005202E0594B5A2B98
:102CCC00800E006E800E5A19005C02E1595100080A
:102CDC0003E3010E506F02D059C150F154B119D019
:102CEC0054A315D0800E5A19006E7F0E005C02E1C1
:102CFC00FC0E595D0BE3800E5A19006E800E4F19B5
:102D0C00005C02E14E51595D01E201D002D0B6EFF8
:102D1C001AF04E514F1106E054A304D0010E4E5F31
:102D2C00000E4F5B4F51000802E14E51080803E2C0
:102D3C00080E506F02D04EC150F155C100F056C173
:102D4C0001F057C102F058C103F0046A056A066A23
:102D5C00076A83EC08F0000ED8A4010E006E005236
:102D6C00D8B453D159C167F1FEEC08F000C004F09F
:102D7C0001C005F002C006F003C007F055C100F019
:102D8C0056C101F057C102F058C103F0BBEC0CF076
:102D9C0000C055F101C056F102C057F103C058F103
:102DAC00010150510008676FFEEC08F000C004F000
:102DBC0001C005F002C006F003C007F055C100F0D9
:102DCC0056C101F057C102F058C103F0BBEC0CF036
:102DDC0000C061F101C062F102C063F103C064F193
:102DEC0061C155F162C156F163C157F164C158F12B
:102DFC0061C100F062C101F063C102F064C103F073
:102E0C0037EC11F0D3EC11F000C004F001C005F068
:102E1C0002C006F003C007F061C100F062C101F00E
:102E2C0063C102F064C103F027EC11F0000E046ED4
:102E3C00000E056E000E066E7E0E076E0CEC0CF08E
:102E4C00000ED8B0010E006E00521AE055C100F011
:102E5C0056C101F057C102F058C103F0000E046EC8
:102E6C00000E056E000E066E7E0E076E64EC06F00C
:102E7C0000C055F101C056F102C057F103C058F122
:102E8C0055C100F056C101F057C102F058C103F012
:102E9C0037EC11F001015051010F096E0A6A000E56
:102EAC000A2209C004F00AC005F0000E0ABEFF0E8B
:102EBC00066E076E04360490053606360736043661
:102ECC000490053606360736560E0424F66E590E57
:102EDC000520F76E000E0620F86E09006F00D4FF77
:102EEC0005F009006F00D4FF06F009006F00D4FF55
:102EFC0007F009006F00D4FF08F00850035C08E1EC
:102F0C000750025C05E10650015C02E10550005CD3
:102F1C001EE3010155C100F056C101F057C102F08A
:102F2C0058C103F0CD0E046ECC0E056E4C0E066E21
:102F3C007B0E076E1FEC02F000C055F101C056F17C
:102F4C0002C057F103C058F1594B5A2B5ED055C1F2
:102F5C0000F056C101F057C102F058C103F037EC34
:102F6C0011F050C104F0000E056E066E076E0436AB
:102F7C0004900536063607360436049005360636B8
:102F8C000736560E0424F66E590E0520F76E000E09
:102F9C000620F86E09006F00D4FF05F009006F00E1
:102FAC00D4FF06F009006F00D4FF07F009006F0092
:102FBC00D4FF08F00850035C08E10750025C05E1FF
:102FCC000650015C02E10550005C1FE2010155C195
:102FDC0000F056C101F057C102F058C103F0000EC9
:102FEC00046E000E056E200E066E820E076E1FEC30
:102FFC0002F000C055F101C056F102C057F103C0F8
:10300C0058F1010E595F000E5A5B010154A393D085
:10301C0054B791D0800E000A006E800E4F19005CE0
:10302C0002E14E510A0804E20A0E4E6F000E4F6F79
:10303C0055C100F056C101F057C102F058C103F060
:10304C0037EC11F000C05BF101C05CF102C05DF126
:10305C0003C05EF15B515C115D115E1142E00A0E22
:10306C00046E000E056E066E076E5BC100F05CC14F
:10307C0001F05DC102F05EC103F018EC0EF008C067
:10308C0000F009C001F00AC002F00BC003F0000E02
:10309C00046E031808E10450021805E104500118ED
:1030AC0002E10050000A1DE1010E4E5F000E4F5B65
:1030BC000A0E046E000E056E066E076E5BC100F004
:1030CC005CC101F05DC102F05EC103F018EC0EF0C2
:1030DC0000C05BF101C05CF102C05DF103C05EF1A8
:1030EC00B9D7800E4F19006E800E005C02E1505172
:1030FC004E5D21E24E51505D676FFEEC08F000C052
:10310C0004F001C005F002C006F003C007F055C181
:10311C0000F056C101F057C102F058C103F0BBECEE
:10312C000CF000C055F101C056F102C057F103C0BC
:10313C0058F14EC150F1050E01014E25006E000EE6
:10314C004F21016E0050515F0150525B4E514F1197
:10315C0003E154B701D004D0010E515F000E525B55
:10316C00030E5315006E54C101F0000E01160050F1
:10317C00011004E0010E515F000E525B53A540D0CC
:10318C0053A315D053A103D02D0E466F02D02B0E96
:10319C00466F6000FFF4E1FF600003F5E2FF6000A2
:1031AC001BF5E6FF3F4B402B5F4B602B0ED053A122
:1031BC000CD06000FFF4E1FF600003F5E2FF200E8D
:1031CC00E66E3F4B402B5F4B602B800E006E800EEB
:1031DC005219005C02E15151000811E26000FFF449
:1031EC00E1FF600003F5E2FF300EE66E3F4B402B33
:1031FC005F4B602B010E515F000E525BE6D741D046
:10320C0053B71AD0800E006E800E5219005C02E18A
:10321C005151000811E26000FFF4E1FF600003F57A
:10322C00E2FF200EE66E3F4B402B5F4B602B010EF6
:10323C00515F000E525BE6D753A315D053A103D0B8
:10324C002D0E476F02D02B0E476F6000FFF4E1FF8D
:10325C00600003F5E2FF60001FF5E6FF3F4B402BDB
:10326C005F4B602B0ED053A10CD06000FFF4E1FF3C
:10327C00600003F5E2FF200EE66E3F4B402B5F4BE8
:10328C00602B55C100F056C101F057C102F058C176
:10329C0003F037EC11F000C05BF101C05CF102C02F
:1032AC005DF103C05EF150C100F0000E016E026EC4
:1032BC00036E00360090013602360336003600905D
:1032CC00013602360336560E0024F66E590E0120D6
:1032DC00F76E000E0220F86E09006F00D4FF04F0A8
:1032EC0009006F00D4FF05F009006F00D4FF06F051
:1032FC0009006F00D4FF07F05BC100F05CC101F066
:10330C005DC102F05EC103F018EC0EF0300E002629
:10331C006000FFF4E1FF600003F5E2FF600003F0E2
:10332C00E6FF3F4B402B5F4B602B4E514F1103E19F
:10333C0054B701D07AD06000FFF4E1FF600003F5D0
:10334C00E2FF2E0EE66E3F4B402B5F4B602B505135
:10335C004E5F000E4F5B505354E0500750C100F0CD
:10336C00000E016E026E036E0036009001360236BE
:10337C00033600360090013602360336560E002412
:10338C00F66E590E0120F76E000E0220F86E090041
:10339C006F00D4FF04F009006F00D4FF05F00900A2
:1033AC006F00D4FF06F009006F00D4FF07F05BC17B
:1033BC0000F05CC101F05DC102F05EC103F018ECDD
:1033CC000EF00A0E046E000E056E066E076E18ECFB
:1033DC000EF008C000F009C001F00AC002F00BC0EA
:1033EC0003F0300E00266000FFF4E1FF600003F5EF
:1033FC00E2FF600003F0E6FF3F4B402B5F4B602B7E
:10340C00AAD74E514F1111E06000FFF4E1FF6000AC
:10341C0003F5E2FF300EE66E3F4B402B5F4B602B0B
:10342C00010E4E5F000E4F5BECD753AB0DD060001E
:10343C00FFF4E1FF600003F5E2FF450EE66E3F4B43
:10344C00402B5F4B602B0CD06000FFF4E1FF600061
:10345C0003F5E2FF650EE66E3F4B402B5F4B602B96
:10346C00800E5A19006E800E005C02E1000E595D50
:10347C0013E259510008596F5A51000E5A57600007
:10348C00FFF4E1FF600003F5E2FF2D0EE66E3F4B0B
:10349C00402B5F4B602B0CD06000FFF4E1FF600011
:1034AC0003F5E2FF2B0EE66E3F4B402B5F4B602B80
:1034BC000A0E046E000E056E59C100F05AC101F0DF
:1034CC009AEC08F0300E00266000FFF4E1FF60007B
:1034DC0003F5E2FF600003F0E6FF01013F4B402BD8
:1034EC005F4B602B0A0E046E000E056E59C100F086
:1034FC005AC101F09AEC08F008C000F009C001F0C4
:10350C00300E00266000FFF4E1FF600003F5E2FFDF
:10351C00600003F0E6FF01013F4B402B5F4B602B3B
:10352C0053A71CD0800E006E800E5219005C02E175
:10353C005151000813E26000FFF4E1FF600003F555
:10354C00E2FF200EE66E3F4B402B5F4B602B010ED3
:10355C00515F000E525B51515211EDE10BEF12F025
:10356C0054A3F7D0800E5A19006E800E005C02E155
:10357C00000E595D0AE2010E595D006E000E5A599B
:10358C00016E00504E5F01504F5B55C100F056C1AB
:10359C0001F057C102F058C103F037EC11F000C034
:1035AC005BF101C05CF102C05DF103C05EF1010E84
:1035BC00506F50510A0A38E050C100F0000E016EF5
:1035CC00026E036E0036009001360236033600366A
:1035DC000090013602360336560E0024F66E590E54
:1035EC000120F76E000E0220F86E09006F00D4FF68
:1035FC0001F009006F00D4FF02F009006F00D4FF46
:10360C0003F009006F00D4FF04F004505E5D08E184
:10361C0003505D5D05E102505C5D02E101505B5DB4
:10362C0001E202D0502BC5D750514E5D656F000E94
:10363C004F59666F65C14EF166C14FF15BC100F029
:10364C005CC101F05DC102F05EC103F0D3EC11F07E
:10365C0000C004F001C005F002C006F003C007F082
:10366C0055C100F056C101F057C102F058C103F02A
:10367C0027EC11F000C061F101C062F102C063F1EE
:10368C0003C064F165C167F1FEEC08F061C104F0A0
:10369C0062C105F063C106F064C107F01FEC02F0D3
:1036AC00000E046E000E056E000E066E7E0E076E8A
:1036BC0064EC06F037EC11F000C05BF101C05CF17A
:1036CC0002C05DF103C05EF14E514F1142E00A0E93
:1036DC00046E000E056E066E076E5BC100F05CC1D9
:1036EC0001F05DC102F05EC103F018EC0EF008C0F1
:1036FC0000F009C001F00AC002F00BC003F0000E8C
:10370C00046E031808E10450021805E10450011876
:10371C0002E10050000A1DE10A0E046E000E056E57
:10372C00066E076E5BC100F05CC101F05DC102F07A
:10373C005EC103F018EC0EF000C05BF101C05CF14F
:10374C0002C05DF103C05EF1010E4E5F000E4F5BD7
:10375C00BBD7800E006E800E4F19005C02E14E51FB
:10376C000C0816E34EC167F18EEC0FF055C104F056
:10377C0056C105F057C106F058C107F064EC06F0CD
:10378C0000C055F101C056F102C057F103C058F109
:10379C0055C100F056C101F057C102F058C103F0F9
:1037AC00046A056A066A076A83EC08F0000ED8A45E
:1037BC00010E006E0052D8B477D055C100F056C13E
:1037CC0001F057C102F058C103F037EC11F0000EB4
:1037DC00046E031808E10450021805E104500118A6
:1037EC0002E10050000A60E1800E006E800E5A1952
:1037FC00005C02E15951010857E259C167F1FEEC36
:10380C0008F000C004F001C005F002C006F003C0CF
:10381C0007F055C100F056C101F057C102F058C174
:10382C0003F0BBEC0CF05F0E046E700E056E090E0F
:10383C00066E810E076E0CEC0CF0010ED8B0000E6B
:10384C00006E005206E0090E0101595F000E5A5B32
:10385C0005D00101080E595F000E5A5B59C167F182
:10386C00FEEC08F000C004F001C005F002C006F048
:10387C0003C007F055C100F056C101F057C102F06A
:10388C0058C103F0BBEC0CF037EC11F000C05BF14D
:10389C0001C05CF102C05DF103C05EF10101556B2A
:1038AC00566B576B586B38D055C100F056C101F0B0
:1038BC0057C102F058C103F037EC11F000C05BF1B6
:1038CC0001C05CF102C05DF103C05EF15BC100F0B0
:1038DC005CC101F05DC102F05EC103F0D3EC11F0EC
:1038EC0000C004F001C005F002C006F003C007F0F0
:1038FC0055C100F056C101F057C102F058C103F098
:10390C0027EC11F000C055F101C056F102C057F17F
:10391C0003C058F1596B5A6B010E506F50510A0A83
:10392C0038E050C100F0000E016E026E036E0036DE
:10393C00009001360236033600360090013602360E
:10394C000336560E0024F66E590E0120F76E000E4B
:10395C000220F86E09006F00D4FF01F009006F001F
:10396C00D4FF02F009006F00D4FF03F009006F00D0
:10397C00D4FF04F004505E5D08E103505D5D05E189
:10398C0002505C5D02E101505B5D01E202D0502B04
:10399C00C5D750514E25006E000E4F21016E595166
:1039AC0000265A5101220050515F0150525B54B70E
:1039BC0004D04E514F1101E104D0010E515F000EA5
:1039CC00525B030E5315006E54C101F0000E01162C
:1039DC000050011004E0010E515F000E525B53A524
:1039EC0040D053A315D053A103D02D0E486F02D055
:1039FC002B0E486F6000FFF4E1FF600003F5E2FF5F
:103A0C00600023F5E6FF3F4B402B5F4B602B0ED045
:103A1C0053A10CD06000FFF4E1FF600003F5E2FF5E
:103A2C00200EE66E3F4B402B5F4B602B800E006EE2
:103A3C00800E5219005C02E15151000811E2600045
:103A4C00FFF4E1FF600003F5E2FF300EE66E3F4B42
:103A5C00402B5F4B602B010E515F000E525BE6D783
:103A6C0041D053B71AD0800E006E800E5219005CF4
:103A7C0002E15151000811E26000FFF4E1FF600027
:103A8C0003F5E2FF200EE66E3F4B402B5F4B602BA5
:103A9C00010E515F000E525BE6D753A315D053A114
:103AAC0003D02D0E496F02D02B0E496F6000FFF42E
:103ABC00E1FF600003F5E2FF600027F5E6FF3F4BF6
:103ACC00402B5F4B602B0ED053A10CD06000FFF449
:103ADC00E1FF600003F5E2FF200EE66E3F4B402B4A
:103AEC005F4B602B50C100F05007005253E050C1A7
:103AFC0000F0000E016E026E036E0036009001366F
:103B0C000236033600360090013602360336560E66
:103B1C000024F66E590E0120F76E000E0220F86E8E
:103B2C0009006F00D4FF04F009006F00D4FF05F00A
:103B3C0009006F00D4FF06F009006F00D4FF07F0F6
:103B4C005BC100F05CC101F05DC102F05EC103F02D
:103B5C0018EC0EF00A0E046E000E056E066E076E63
:103B6C0018EC0EF008C000F009C001F00AC002F019
:103B7C000BC003F0300E00266000FFF4E1FF600084
:103B8C0003F5E2FF600003F0E6FF3F4B402B5F4B79
:103B9C00602BA8D7800E006E800E5A19005C02E1D3
:103BAC005951000811E26000FFF4E1FF600003F5D9
:103BBC00E2FF300EE66E3F4B402B5F4B602B010E4D
:103BCC00595F000E5A5BE6D7800E000A006E800E1D
:103BDC004F19005C02E14E51080803E2080E506FC9
:103BEC0002D04EC150F150514E5F000E4F5B5053FE
:103BFC0003E154B701D00CD06000FFF4E1FF60008A
:103C0C0003F5E2FF2E0EE66E3F4B402B5F4B602B15
:103C1C0050C167F1FEEC08F055C104F056C105F037
:103C2C0057C106F058C107F01FEC02F07FEC0DF005
:103C3C0000C05BF101C05CF102C05DF103C05EF13C
:103C4C00505354E0500750C100F0000E016E026E4C
:103C5C00036E0036009001360236033600360090B3
:103C6C00013602360336560E0024F66E590E01202C
:103C7C00F76E000E0220F86E09006F00D4FF04F0FE
:103C8C0009006F00D4FF05F009006F00D4FF06F0A7
:103C9C0009006F00D4FF07F05BC100F05CC101F0BC
:103CAC005DC102F05EC103F018EC0EF00A0E046E5A
:103CBC00000E056E066E076E18EC0EF008C000F0D4
:103CCC0009C001F00AC002F00BC003F0300E002650
:103CDC006000FFF4E1FF600003F5E2FF600003F019
:103CEC00E6FF3F4B402B5F4B602BAAD74E514F1139
:103CFC0011E06000FFF4E1FF600003F5E2FF300E1D
:103D0C00E66E3F4B402B5F4B602B010E4E5F000E5F
:103D1C004F5BECD753A71CD0800E006E800E52194F
:103D2C00005C02E15151000813E26000FFF4E1FF76
:103D3C00600003F5E2FF200EE66E3F4B402B5F4B1D
:103D4C00602B010E515F000E525B51515211EDE18F
:103D5C000BEF12F0C00E5315016E54C102F0000EA1
:103D6C000216000E021802E1000E0118D8A49ED013
:103D7C0053A937D0600013F5E9FF600017F5EAFF8F
:103D8C006F00B8FF00F06F00B8FF01F0600003F0A7
:103D9C00E9FF600007F0EAFF6F00B8FF5BF16F000E
:103DAC00B8FF5CF16F00B8FF5DF16F00B8FF5EF11A
:103DBC00600013F5E9FF600017F5EAFF040EEE242E
:103DCC00006E000EEE20016E600013F5E1FF600046
:103DDC0017F5E2FF600003F0E6FF600007F0E6FF76
:103DEC003DD0600013F5E9FF600017F5EAFF6F00A6
:103DFC00B8FF00F06F00B8FF01F0600003F0E9FFBE
:103E0C00600007F0EAFF6F00B8FF00F06F00B8FF2A
:103E1C0001F0000E01BEFF0E026E036E00C05BF1DE
:103E2C0001C05CF102C05DF103C05EF1600013F5EE
:103E3C00E9FF600017F5EAFF020EEE24006E000E9B
:103E4C00EE20016E600013F5E1FF600017F5E2FF54
:103E5C00600003F0E6FF600007F0E6FF800E5E19DD
:103E6C00006E800E005C08E1000E5D5D05E1000E49
:103E7C005C5D02E1000E5B5D18E2030E5313000E55
:103E8C005413006A016A026A036A5B51005E5C515A
:103E9C00015A5D51025A5E51035A00C05BF101C0D8
:103EAC005CF102C05DF103C05EF16CD053A937D058
:103EBC00600013F5E9FF600017F5EAFF6F00B8FF2B
:103ECC0000F06F00B8FF01F0600003F0E9FF600044
:103EDC0007F0EAFF6F00B8FF5BF16F00B8FF5CF111
:103EEC006F00B8FF5DF16F00B8FF5EF1600013F575
:103EFC00E9FF600017F5EAFF040EEE24006E000ED9
:103F0C00EE20016E600013F5E1FF600017F5E2FF93
:103F1C00600003F0E6FF600007F0E6FF33D06000BE
:103F2C0013F5E9FF600017F5EAFF6F00B8FF00F02A
:103F3C006F00B8FF01F0600003F0E9FF600007F0CC
:103F4C00EAFF6F00B8FF5BF16F00B8FF5CF1000E89
:103F5C005D6F5E6F600013F5E9FF600017F5EAFF17
:103F6C00020EEE24006E000EEE20016E600013F5C2
:103F7C00E1FF600017F5E2FF600003F0E6FF600070
:103F8C0007F0E6FF000E4F1902E1000E4E190FE18B
:103F9C00000E006E5E1908E100505D1905E100503D
:103FAC005C1902E15B51000A02E14E4B4F2BC00E33
:103FBC005315006E00C005F0BAD0010E506F505171
:103FCC000A0A38E050C100F0000E016E026E036E5A
:103FDC00003600900136023603360036009001366A
:103FEC0002360336560E0024F66E590E0120F76E7B
:103FFC00000E0220F86E09006F00D4FF01F00900DA
:10400C006F00D4FF02F009006F00D4FF03F0090029
:10401C006F00D4FF04F004505E5D08E103505D5D59
:10402C0005E102505C5D02E101505B5D01E202D0F2
:10403C00502BC5D78BD0010E506F5051080A38E069
:10404C0050C100F0000E016E026E036E003600903F
:10405C00013602360336003600900136023603363E
:10406C00590E0024F66E5A0E0120F76E000E022037
:10407C00F86E09006F00D4FF01F009006F00D4FF47
:10408C0002F009006F00D4FF03F009006F00D4FFA9
:10409C0004F004505E5D08E103505D5D05E10250E3
:1040AC005C5D02E101505B5D01E202D0502BC5D793
:1040BC004DD0010E506F50510C0A38E050C100F039
:1040CC00000E016E026E036E003600900136023651
:1040DC000336003600900136023603367B0E002480
:1040EC00F66E580E0120F76E000E0220F86E0900D5
:1040FC006F00D4FF01F009006F00D4FF02F009003B
:10410C006F00D4FF03F009006F00D4FF04F00450DB
:10411C005E5D08E103505D5D05E102505C5D02E10E
:10412C0001505B5D01E202D0502BC5D70FD005507A
:10413C00000AD8B442D70550C00AD8B43ED70550AF
:10414C00800AD8B478D70550400AB3E0800E006ED0
:10415C00800E4F19005C02E14E51505D03E24EC1DE
:10416C0050F10DD0800E4F19006E800E005C02E1F4
:10417C0050514E5D04E250C14EF1000E4F6F515143
:10418C0052110EE0030E5315006E54C101F0000ED7
:10419C0001160050011004E0010E515F000E525B3D
:1041AC00800E4F19006E800E5219005C02E15151C5
:1041BC004E5D05E24E51515F4F51525B02D0516B37
:1041CC00526BC40E5315016E5451080B026E025003
:1041DC00080A02E1400E011808E15151521104E0A5
:1041EC00010E515F000E525B1CD0C00E5315016EB8
:1041FC005451080B026E0250080A02E1800E01189D
:10420C0010E1800E006E800E5219005C02E15151DB
:10421C00020805E2020E515F000E525B02D0516B98
:10422C00526B53A569D053A315D053A103D02D0EB7
:10423C004A6F02D02B0E4A6F6000FFF4E1FF600062
:10424C0003F5E2FF60002BF5E6FF3F4B402B5F4B85
:10425C00602B3BD053A10DD06000FFF4E1FF600058
:10426C0003F5E2FF200EE66E3F4B402B5F4B602BBD
:10427C002CD0C00E5315016E5451080B026E025017
:10428C00080A02E1800E011820E16000FFF4E1FF52
:10429C00600003F5E2FF300EE66E3F4B402B5F4BA8
:1042AC00602B53AB03D0580E4B6F02D0780E4B6F74
:1042BC006000FFF4E1FF600003F5E2FF60002FF502
:1042CC00E6FF3F4B402B5F4B602B5151521113E0DB
:1042DC006000FFF4E1FF600003F5E2FF300EE66ED4
:1042EC003F4B402B5F4B602B010E515F000E525B1E
:1042FC0051515211EDE182D05151521115E053B789
:10430C0013D06000FFF4E1FF600003F5E2FF200E24
:10431C00E66E3F4B402B5F4B602B010E515F000E46
:10432C00525B51515211EDE153A315D053A103D05F
:10433C002D0E4C6F02D02B0E4C6F6000FFF4E1FF82
:10434C00600003F5E2FF600033F5E6FF3F4B402BC6
:10435C005F4B602B0ED053A10CD06000FFF4E1FF3B
:10436C00600003F5E2FF200EE66E3F4B402B5F4BE7
:10437C00602BC00E5315016E5451080B026E025087
:10438C00080A02E1400E01180DE16000FFF4E1FFA4
:10439C00600003F5E2FF300EE66E3F4B402B5F4BA7
:1043AC00602B2CD0C00E5315016E5451080B026EAD
:1043BC000250080A02E1800E011820E16000FFF4AF
:1043CC00E1FF600003F5E2FF300EE66E3F4B402B41
:1043DC005F4B602B53AB03D0580E4D6F02D0780E51
:1043EC004D6F6000FFF4E1FF600003F5E2FF600039
:1043FC0037F5E6FF3F4B402B5F4B602B800E006E7A
:10440C00800E4F19005C02E14E51505D0DE26000D0
:10441C00FFF4E1FF600003F5E2FF300EE66E3F4B68
:10442C00402B5F4B602BEAD74EC100F04FC101F01F
:10443C00010E4E5F000E4F5B00500110D8B43FD1FF
:10444C00C00E5315006E00C061F11CD14EC100F0BE
:10445C004FC101F0000E4FBFFF0E026E036E00360F
:10446C0000900136023603360036009001360236D3
:10447C000336560E0024F66E590E0120F76E000E10
:10448C000220F86E09006F00D4FF04F009006F00E1
:10449C00D4FF05F009006F00D4FF06F009006F008F
:1044AC00D4FF07F05BC100F05CC101F05DC102F00C
:1044BC005EC103F018EC0EF00A0E046E000E056ED1
:1044CC00066E076E18EC0EF008C000F009C001F083
:1044DC000AC002F00BC003F0300E0024506FE1D084
:1044EC0053AB4AD04EC100F04FC101F0000E4FBF8C
:1044FC00FF0E026E036E0036009001360236033654
:10450C0000360090013602360336590E0024F66E42
:10451C005A0E0120F76E000E0220F86E09006F0093
:10452C00D4FF04F009006F00D4FF05F009006F0000
:10453C00D4FF06F009006F00D4FF07F05BC100F058
:10454C005CC101F05DC102F05EC103F018EC0EF02D
:10455C000F0E0016000E011602160316390E00245B
:10456C00F66E5B0E0120F76E000E0220F86E09004D
:10457C006F00D4FF50F149D04EC100F04FC101F093
:10458C00000E4FBFFF0E026E036E00360090013618
:10459C000236033600360090013602360336590EC9
:1045AC000024F66E5A0E0120F76E000E0220F86EF3
:1045BC0009006F00D4FF04F009006F00D4FF05F070
:1045CC0009006F00D4FF06F009006F00D4FF07F05C
:1045DC005BC100F05CC101F05DC102F05EC103F093
:1045EC0018EC0EF00F0E0016000E01160216031634
:1045FC00280E0024F66E5B0E0120F76E000E0220D2
:10460C00F86E09006F00D4FF50F14BD04EC100F092
:10461C004FC101F0000E4FBFFF0E026E036E00364D
:10462C000090013602360336003600900136023611
:10463C0003367B0E0024F66E580E0120F76E000E2A
:10464C000220F86E09006F00D4FF04F009006F001F
:10465C00D4FF05F009006F00D4FF06F009006F00CD
:10466C00D4FF07F05BC100F05CC101F05DC102F04A
:10467C005EC103F018EC0EF0070E0014506F300EF4
:10468C0050270FD06151000AD8B4E0D66151C00A4E
:10469C00D8B4DCD66151800AD8B422D76151400A13
:1046AC00B5E06000FFF4E1FF600003F5E2FF60009D
:1046BC0043F5E6FF3F4B402B5F4B602BB5D653A722
:1046CC001CD0800E006E800E5219005C02E151511C
:1046DC00000813E26000FFF4E1FF600003F5E2FF65
:1046EC00200EE66E3F4B402B5F4B602B010E515F53
:1046FC00000E525B51515211EDE10BEF12F05FC104
:08470C0000F060C101F0120091
:0C4714006F00A0F701F001C000F01200DF
:104720003FC121F140C122F141C123F142C124F135
:1047300043C11DF144C11EF145C11FF146C120F125
:1047400047C10FF148C110F149C111F14AC112F13D
:104750004BC113F14CC114F14DC115F14EC116F10D
:02476000120045
:10476200FC0E3F015E175E81010EAE6E7C6A7D6AB1
:02477200120033
:10477400FE0E0101196F470E1A6F3F0E1B6F010EDB
:104784001C6F3E01F86BF96BFA6BFB6BEC0EFD17BB
:08479400F889F885F88F120086
:10479C00160E0101676F686B130E696F2BEC11F02D
:1047AC00170E0101676F010E686F250E696F2BECF8
:0447BC0011F01200E6
:1047C0000101426B6000FFF4E9FF600003F5EAFFBE
:1047D0006F00B8FF41F14151000A10E041C167F19B
:1047E000ABEC0CF00101422B42513F25E96E000E6B
:0E47F0004021EA6E6F00B8FF41F1EDD71200D4
:1047FE003F0E01013F153E01F16F79EC0DF0F8818E
:10480E000000F8A101D0FDD76F00BCFB00F06F00D7
:06481E00C0FB01F01200D6
:104824007E982FC100F0016A600003F07DFFFF0E47
:0848340001012E157C6E12003B
:0C483C002EC13FF12FC140F1BDDF120082
:104848000D0E0101706F17EC01F00A0E0101706F77
:0648580017EC01F0120054
:10485E00330E01013D6F010E3E6F2EC13FF12FC190
:10486E0040F130C141F131C142F132C143F13D0E4F
:10487E00446F010E456F06EC12F000C03BF101C013
:10488E003CF100502E25E16E01502F21E26EE66ABA
:0A489E003BC100F03CC101F0120024
:1048A8006000BBF4E9FF6000BFF4EAFFEE5215E0D8
:1048B8006000BBF4E9FF6000BFF4EAFF6000C3F4E6
:1048C800D9FF6000C7F4DAFFEE50DE1806E10101F7
:1048D8002E4B2F2B304B312BE3D76000BBF4E9FF75
:1048E8006000BFF4EAFF6000C3F4D9FF6000C7F4BA
:1048F800DAFFDE50EE5C006E016A000E015A12000B
:0449080005DF1200B5
:0A490C00AC8E7E8E0C0E7E1212009F
:104916006000BBF4F6FF6000BFF4F7FF6000C3F46D
:10492600F8FF09006F00D4FF00F0005216E06000A7
:10493600BBF4F6FF6000BFF4F7FF6000C3F4F8FFB6
:1049460009006F00D4FF70F117EC01F0010E0101B0
:0C4956002E27000E2F233023DBD7120089
:0C49620008DF2EC13FF14ADFF89F120071
:04496E00F9DE12005C
:10497200120E0101676F686B090E696F2BEC11F063
:04498200EFDE120052
:1049860009006F00D7FFE6FF0006FAE10106F8E12D
:0249960012000D
:104998002EC102F02FC103F002C000F003C001F0E5
:1049A800024A032A600003F0E9FF600007F0EAFF0B
:1049B800EE5201E0F1D701012E51025C006E2F5139
:0E49C8000358016E010E005E000E015A12002F
:1049D6003901C06BC16BC26BFF0ECA6E3A01406BE8
:1049E6004083830EC26E41934293C296C298C2948C
:1049F600BA86BA88BA84506BCB6AFF0EC36EFF0EB6
:104A0600516F3E01BC6BB86BCC6A920EC46E3A0114
:104A1600606B130E166F170EE56FC490BC903E01C7
:0A4A2600C16BC19FC183C191120052
:104A3000AB50010F006E016A000E01222EC104F07E
:104A40002FC105F07FEC0CF0060E046E00C002F0E2
:104A500001C003F0045005E003320232039EFF0F51
:104A6000FAD760000BF07CFF60000FF07DFF1200B2
:104A70003F6A406A000E405C02E14F0E3F5C18E264
:104A8000430E3F24E16E000E4020E26E6F0087FF70
:104A9000E1FF6F008BFFE2FFE66A010E3F24006E2C
:104AA000000E4020016E00C03FF001C040F0E2D790
:104AB000436A3F6A406A416A426A366A376A346AC0
:104AC000356A386A3D01F289F96BFA6B39019387CF
:024AD0001200D2
:104AD20064DE080E01013F6F490E406F000E416F08
:104AE200000E426F2E0E436F020E446F700E456F22
:104AF200010E466FFF0E476FFF0E486F000E496FA3
:104B0200000E4A6FB00E4B6F010E4C6F000E4D6FD0
:104B1200000E4E6F04DE3F6B406BE6EC11F01200AC
:104B22006000BBF4E9FF6000BFF4EAFF6F00B8FF6A
:104B320030F1000E0101316F000E316F000E31199C
:104B420002E1200E301907E0000E311902E1090ED0
:104B5200301901E003D02E4B2F2BE2D7326B336B8F
:104B6200346B356B000E311902E12D0E301905E15F
:104B7200344B352B2E4B2F2B08D0000E311902E16E
:104B82002B0E301902E12E4B2F2B6000BBF4E9FFF4
:104B92006000BFF4EAFF6F00B8FF30F1000E316F22
:104BA200000E316F30C167F173EC0CF0005219E066
:104BB20032C100F033C101F00A0E046E000E056E20
:104BC2007FEC0CF0300E305D026E000E3159036E38
:104BD20002500024326F03500120336F2E4B2F2BD3
:104BE200D4D73451351108E032510008006E33C178
:104BF20001F0000E015604D032C100F033C101F0C1
:024C020012009E
:104C0400B3EC2DF0600E3901D96F060EDF6FE1DED3
:104C14000001E76BE86B000EE85D02E1200EE75D42
:104C240010E2E90EE725E16E000EE821E26E6F0066
:104C340087FFE1FF6F008BFFE2FFE66AE74BE82B9B
:104C4400EAD7E76BE86B000EE85D02E1500EE75D22
:104C540010E2970EE725E16E000EE821E26E6F0088
:104C640087FFE1FF6F008BFFE2FFE66AE74BE82B6B
:104C7400EAD73F6A406A366A376A970E936F000E26
:104C8400946FA00E3D01F56F010EF66FF28F1FDFDA
:104C9400080E01013F6F490E406F000E416F000E78
:104CA400426F2E0E436F020E446F700E456F010E5D
:104CB400466FFF0E476FFF0E486F000E496F000EE0
:104CC4004A6FB00E4B6F010E4C6F000E4D6F000E0D
:104CD4004E6F24DD090E0B6E1E0E0C6EE40E0D6E6F
:104CE4000D2EFED70C2EFCD70B2EFAD700000C0E7F
:104CF400706F17EC01F0A6DD050E01012E6F5B0E3F
:104D04002F6F000E306F05DEF10E01012E6F5A0E6B
:104D14002F6F000E306FFDDD940E01012E6F560EC5
:104D24002F6F000E306FF5DD0E0E01012E6F560E43
:104D34002F6F000E306FEDDD530E01012E6F560EF6
:104D44002F6F000E306FE5DD4B0E01012E6F580EF4
:104D54002F6F000E306FDDDD170E01012E6F5B0E1D
:104D64002F6F000E306FD5DD000E0001956F7D0EA4
:104D7400966F93C02EF194C02FF1380E0101306F5D
:104D84005A0E316F000E326F000E336F7D0E346F8A
:104D940064DD93C02EF194C02FF14EDDCC0E2E6F46
:104DA400590E2F6F000E306FB4DDCF0E01012E6F40
:104DB400560E2F6F000E306FACDD090E01012E6F01
:104DC400570E2F6F000E306FA4DD7B0E01012E6F86
:104DD400570E2F6F000E306F9CDD040E01012E6FF5
:104DE400590E2F6F000E306F94DDC50E01012E6F2A
:104DF4005A0E2F6F000E306F8CDD040E01010B6F05
:104E0400000E0C6F000E006E0C51005C02E10B51A1
:104E1400000823E2BC840D0E0B6E2D0E0C6ED70E13
:104E24000D6E0D2EFED70C2EFCD70B2EFAD70000DC
:104E34000000BC940D0E0B6E2D0E0C6ED70E0D6E75
:104E44000D2EFED70C2EFCD70B2EFAD70000000037
:104E5400010E0B5F000E0C5BD5D78ADC010E01013D
:104E64002E6F7DDD00C00DF101C00EF101010A9528
:104E74001F6A206AD28ED28C3901938F0001E76BAE
:104E8400E86B0101096B170E2E6F5A0E2F6F000E7F
:104E9400306F3FDDD80E01012E6F580E2F6F000EBC
:104EA400306F37DD1FEC01F0090E126F10EC01F0CA
:104EB400F20E01012E6F590E2F6F000E306F29DD97
:104EC400800E1D6E000E1E6E500EAC12F90EAB6EEF
:104ED4004EDD500EAC12F90EAB6E47DD15DD1DC074
:104EE4002EF11EC02FF1A2DDADDC3F6A406A366AA6
:104EF400376A346A356A3901818B918BD28E396A6B
:104F04003A6A970E0001936F000E946FE76BE86B9B
:104F14003B6A3C6AABDD520E0B6E2B0E0C6E000E20
:104F24000D6E0D2EFED70C2EFCD70B2EFAD70000DB
:104F3400010E01012E6F13DD00C03DF001C03EF0F3
:104F44001C50000A44E12D50000A16E13DC01DF03A
:104F54003EC01EF01E321D321E9E1E321D321E9E8B
:104F64001E321D321E9E1E321D321E9E080E01016F
:104F7400276F000E286F0FD001013DC01DF03EC009
:104F84001EF01E321D321E9E1E321D321E9E0A0E41
:104F9400276F000E286F93C02EF194C02FF1700E6E
:104FA400306F550E316F000E326F3BC033F13CC091
:104FB40034F13DC035F13EC036F127C137F128C187
:104FC40038F11DC039F11EC03AF147DC25D02D500F
:104FD400000A06E10101080E276F000E286F05D0B4
:104FE40001010A0E276F000E286F93C02EF194C0A2
:104FF4002FF1C20E306F550E316F000E326F3BC071
:1050040033F13CC034F127C135F128C136F11DC05C
:1050140037F11EC038F121DC93C02EF194C02FF17A
:105024000BDC800E006E800E3A18005C02E13950F1
:10503400000815E293C02EF194C02FF14A0E306F90
:105044005B0E316F000E326F39C033F13AC034F168
:1050540004DC93C02EF194C02FF11EEC24F024EC58
:1050640024F0000E351802E1010E3418D8A446D2FB
:10507400970E0001936F000E946F93C02EF194C0AD
:105084002FF1DC0E0101306F5A0E316F000E326FBA
:10509400430E336F000E346F2FEC24F093C02EF1C7
:1050A40094C02FF11EEC24F04350430AD8A4C3D07B
:1050B400000E006E3750005C02E136500108D8B093
:1050C400BAD00101440E2E6F000E2F6F63DC00C0B6
:1050D40025F101C026F1010E0001E76F000EE86F13
:1050E400010126510001E85D04E10101255100019F
:1050F400E75D1DE2430EE725E96E000EE821EA6E46
:105104006F00A7FFE9FF6F00ABFFEAFF6F00B8FF76
:1051140000F000C029F129C167F173EC0CF00050D4
:10512400000A01E104D00001E74BE82BD9D70001C4
:10513400E8510101261903E125510001E719D8A41A
:1051440078D0440E01012E6F000E2F6FE8DC00C0F2
:1051540025F101C026F12D50000A0FE1000E006E6A
:105164002651005C02E12551000807E2010E265D8C
:1051740002E1000E255D01E213D02D50010A0FE17A
:10518400000E006E2651005C02E12551000807E282
:10519400040E265D02E1000E255D01E201D005D07A
:1051A40025C11DF026C11EF002D01D6A1E6A2D50B5
:1051B400000A1CE10101080E276F000E286F1DC0B4
:1051C4002EF1000E2F6F32DC93C02EF194C02FF11C
:1051D4007E0E0101306F590E316F000E326F1DC00B
:1051E40033F11EC034F12FEC24F01BD001010A0E60
:1051F400276F000E286F1DC02EF11EC02FF112EC78
:1052040024F093C02EF194C02FF12D0E306F590E5F
:10521400316F000E326F1DC033F11EC034F12FEC1C
:1052240024F093C02EF194C02FF11EEC24F0010E53
:105234001C6E0101296B0101430E2E6F000E2F6FAE
:105244002E0E306F000E316F54EC24F000C02CF1A0
:1052540001C02DF1000E011802E1000E0018D8A4BF
:10526400D2D0000E351802E1010E3418D8A4CBD0E8
:105274002D50000A2AE10101256B266B000E265DE4
:1052840002E1F00E255D20E225C12AF126C12BF1B1
:10529400080E276F000E286F25C12EF126C12FF1AD
:1052A40018EC25F0110E0B6E3C0E0C6ECB0E0D6E31
:1052B4000D2EFED70C2EFCD70B2EFAD7100E0101A3
:1052C4002527000E2623DAD728D00101256B266B6B
:1052D400030E265D02E1BF0E255D1FE225C12AF102
:1052E40026C12BF10A0E276F000E286F25C12EF15F
:1052F40026C12FF112EC24F0110E0B6E3C0E0C6E35
:10530400CB0E0D6E0D2EFED70C2EFCD70B2EFAD71E
:10531400400E2527000E2623DBD72D50000A2DE151
:10532400FF0E256F000E266F000E006E2651005CE6
:1053340002E12551100820E225C12AF126C12BF1F2
:10534400080E276F000E286F25C12EF126C12FF1FC
:1053540018EC25F0110E0B6E3C0E0C6ECB0E0D6E80
:105364000D2EFED70C2EFCD70B2EFAD7100E0101F2
:10537400255F000E265BD8D72BD0FC0E256F030EBD
:10538400266F000E006E2651005C02E12551400894
:105394001FE225C12AF126C12BF10A0E276F000E48
:1053A400286F25C12EF126C12FF112EC24F0110E25
:1053B4000B6E3C0E0C6ECB0E0D6E0D2EFED70C2E0E
:1053C400FCD70B2EFAD7400E255F000E265BD9D7EB
:1053D4002D50000A0BE1080E276F000E286F1DC028
:1053E4002EF11EC02FF118EC25F00BD00A0E01018E
:1053F400276F000E286F1DC02EF11EC02FF112EC76
:1054040024F0346A356A4350410A0BE1000E006E01
:105414003750005C02E13650000803E2346A356A12
:105424001C6A4350500A1DE1000E006E3750005CA8
:1054340002E13650000815E2346A356A4450310AF4
:1054440008E101010A0E276F000E286F010E2D6E70
:1054540006D00101080E276F000E286F2D6A346AEA
:10546400356A0101430E2E6F000E2F6F280E306F28
:10547400000E316F54EC24F000C02CF101C02DF16A
:10548400000E011802E1000E001838E1590E010166
:105494002E6F5B0E2F6F000E306F8BEC24F0190E05
:1054A40001012E6F580E2F6F000E306F8BEC24F01D
:1054B400420E01012E6F570E2F6F000E306F8BECD2
:1054C40024F0AB0E01012E6F580E2F6F000E306FBB
:1054D4008BEC24F0A50E01012E6F590E2F6F000ED8
:1054E400306F8BEC24F0AE0E01012E6F5A0E2F6F2D
:1054F400000E306F8BEC24F0346A356A000E3518D8
:1055040002E1020E34181EE1970E0001936F000EA3
:10551400946F93C02EF194C02FF1790E0101306F76
:105524005A0E316F000E326F36C033F137C034F18A
:105534002FEC24F093C02EF194C02FF11EEC24F034
:1055440038EC25F02D50000A07E11DC02EF11EC0D5
:105554002FF118EC25F006D01DC02EF11EC02FF13E
:0C55640012EC24F03B4A3C2AD5D4FFD7BF
:105B660010EE1CF0180E006E010E016E960EF66E0B
:0E5B76005A0EF76E000EF86EC3EC24F012000B
:10557000204D6573757265202325356420205265A2
:10558000676C6167652044757479202076696120B5
:105590004144432F20524131203D3E202520356497
:1055A00020204D6F64652050574D202532642062C5
:1055B000697473202049526174696F203D2530342D
:0255C000640085
:1055C200204D657375726520232535642020526550
:1055D200676C616765207669612063646520436C4E
:1055E200617669657220437878787820204D6F64FF
:1055F200652050574D202532642062697473202043
:0C5602002049526174696F3D2535640039
:10560E002050726F6A6574203A2031384632374B1B
:10561E0034325F55415254315F52585F49545F41A5
:10562E004443305F50574D315F38625F3130625FB7
:10563E00426173655F323032325F30382E6D637087
:05564E0070690D0A0067
:1056530020536F75726365203A205F3138463237C5
:105663004B34325F33324D687A5F55617274315F08
:105673004144435F50574D5F38625F6F755F313010
:10568300625F5F323032325F303831322E630D0A5F
:015693000016
:10569400204469726563746F7279203A20433A5CDE
:1056A4005F4D696B726F435C5F4D657350726F6AD7
:1056B4006574735F4D696B726F435C5F313846325A
:0B56C400374B34325F50574D0D0A0089
:1056CF00204378787820706F7572207361697369E1
:1056DF00652056616C6575722078787878204475EE
:1056EF007479202050574D20766961206C652043D6
:0A56FF006C6176696572200D0A00E7
:10570900204120706F75722056616C657572204456
:105719007574792050574D206973737565206475C8
:1057290020506F746172202F52413120416E616C9B
:095739006F67697175650D0A00C6
:10574200204120706F75722056616C65757220441D
:105752007574792050574D2069737375652064758F
:1057620020506F746172202F52413120416E616C62
:095772006F67697175650D0A008D
:10577B0020503120706F7572206D6F64652050570B
:10578B004D20313062697473202C202050302070F2
:10579B006F7572206D6F64652050574D20382062F5
:0657AB006974730D0A0091
:1057B1000000007FCDCC4C7B0AD723786F12037594
:1057C10017B75171ACC5276EBD37066B95BF5667CC
:1057D10077CC2B645F700961FFE65B5D08E53C3CBB
:0457E1006042221BE5
:1057E5000000007F000020820000488500007A88C4
:1057F50000401C8C0050438F0024749280961896AC
:1058050020BC3E99286B6E9CF90215A0EC782DC141
:04581500CAF249E2A8
:10581900204320706F757220736169736965205622
:10582900616C6575722044757479202050574D203C
:10583900766961206C6520436C6176696572200D1B
:025849000A0053
:10584B0020434F4E464947203A2050313846323795
:10585B004B34325F464F53435F51384D487A78345F
:10586B005F33324D487A2E6366677363680D0A00A7
:10587B0001000000080000004000000000020000D2
:10588B000010000000800000000004000000200059
:10589B0000000001000000080000004000000000B4
:1058AB0020503120706F7572206D6F646520313020
:1058BB0062697473202020503020706F7572206DD8
:0D58CB006F6465203820626974730D0A0057
:1058D800204166666563746174696F6E2028505054
:1058E80053292050494E2052433220E020536F72F2
:0C58F8007469652050574D31200D0A00E6
:105904002052414D504520706F75722072616D7048
:1059140065205570202C20707569732052616D705C
:095924006520446F776E0D0A0046
:10592D002050574D206D6F64653D203130206269E8
:10593D00747320204E65772049526174696F202061
:09594D003D20253564200D0A00FF
:10595600010000000A00000064000000E8030000E7
:1059660010270000A086010040420F008096980094
:0859760000E1F50500CA9A3BAF
:10597E002050574D206D6F6465203D20386269744C
:10598E007320204E65772049526174696F203D2047
:07599E00253564200D0A000D
:1059A5002052414D504520706F75722072616D70A7
:1059B5006520557020707569732052616D70652082
:0759C500446F776E0D0A002C
:1059CC000D0A20436F6D6D616E64652076696120F0
:1059DC004B6579626F617264205465726D696E619A
:0659EC006C203A0D0A00D8
:1059F20020496E69742050574D31203862697473A2
:105A02002061742031303030487A206F6E2052434A
:055A120032200D0A0026
:105A1700205573616765206465206C61204C69625D
:105A2700726169726965204D696B726F43200D0A57
:015A3700006E
:105A380020436C6F636B20696E697469616C6520C3
:105A4800696E204B687A203D2025303575200D0A77
:015A5800004D
:105A5900010000001000000000010000001000001B
:105A6900000001000000100000000001000000100B
:105A7900427566666572312055415254312046752A
:0D5A89006C6C203D2025303564200D0A0096
:015A9600000F
:025A970000000D
:025A990000000B
:075A9B00286E756C6C2900F8
:055AA20048656C700076
:015AA70000FE
:065AA80052414D50450083
:105AAE002048656C70203A206365747465206169C6
:075ABE0064650D0A0D0A00EA
:105AC5002048656C70203A206365747465206169AF
:075AD50064650D0A0D0A00D3
:105ADC00205265636570742055415254313D202528
:055AEC0073200D0A000B
:105AF10020506F77657220737570706C793A20351C
:045B0100560D0A0033
:105B0500204D4355203A2031384632374B34320D3B
:025B15000A0084
:105B170020464F534320203A2033324D487A0D0A0E
:015B2700007D
:105B2800303132333435363738396162636465660B
:015B3800006C
:105B390030313233343536373839414243444546BA
:015B4900005B
:0F5B4A002020657272657572203D20253564003C
:0C5B59000D0A2048656C70203A0D0A000F
:020000040030CA
:0A000000040927A70B3F9F0F010022
:00000001FF
